:2000000002002632000000000000004390E943B030C28C32000000000000003200000000F5
:200020000000000201F0758122758921758DFF75884075987CC2AFD2ACD2A9D2BC7590FFD3
:2000400075B0FF7509017508007521007F00750B0075200075B07F1201E775B0FF7590FD92
:200060001201E77590FB1201E77590EF1201E775907F1201E77590BF1201E77590DF12016B
:20008000E77590F71201E77590FF75B0EF1201E775B0DF1201E775B0FF7590FE1201E775DD
:2000A00090FF75B0DF1201E775B0EF1201E775B0FF7590F71201E77590DF1201E77590BFE9
:2000C0001201E775907F1201E77590FF1201E71201E71201E7C299C298D2AF20B319D20CB6
:2000E0007590FF75B0FF300EFD758CD8758AEFC297D28CC20E80EF20B208D20A30B2FD1239
:2001000001E7120151300E0312019B12011312013280EF30B20720090122C209221201E7AE
:2001200020090ED209E509B40305750900800205092230B30720080122C208221201E72098
:20014000080ED208E509B400057509038002150922E509B5080122850908E508B4000D4370
:20016000901643B080C294750A03802BB4010D43901643B080C292750A04801BB4020D434D
:20018000901643B080C291750A05800BB40308439016C2B7750A07750B0022758C8A758A11
:2001A000CF300A0879147870D8FED9FCE50BB50A04750B00E47004C2978025147004C296A5
:2001C000801E147004C2958017147004C2938010147004C2B48009147004C2B58002C29044
:2001E000D28C050BC20E22793B7859D8FED9FC22C2AFC0D0C0E0859920E520300C04D20E49
:200200008038B4F80D300D320FBF182ED20E7F008028401CB4FA0BD20DD20E750B007F0010
:200220008018B4FB04D20D8011B4FC0EC20D800A200F1474CFB5200BD20FD0E0D0D0C298FB
:20024000D2AF32C20F80F32007E9E520B404005004F50980E5B47F02D20AB47EDDC20A80B7
:20026000D92B2B2B204D494449204265617456696577657220322056312E3031202F20419B
:200280005438394332303531202F202843292053746566616E204861726173696D2030389D
:0902A0002F32303037202B2B2BBC
:0002A90154
